:100808002025322E5820002053797374656D2048B6
:10081800414C54454400204C6F632E20537465703E
:10082800706572206572726F7200205379737465F7
:100838006D20524553455400202E2E2E2E204372F3
:10084800656174696E672072616D702000202E2EBC
:100858002E2E2E2046696E652061646A7573742099
:1008680020002044652D53796E6368726F6E697A33
:100878006564202000496E697420536C696465734F
:10088800202E2E2E002020202E2E2E20506C65612A
:100898007365207761697400204D656368616E69CE
:1008A80063616C204572726F72002020202E2E2EFC
:1008B8002053796E6368726F6E697A6564002E2EB4
:1008C8002E4F766572666C6F7720746F204D494E97
:1008D8002020002E2E2E556E646572666C6F772070
:1008E800746F204D415820002E2E2E416476616E83
:1008F800636520746F2025342E64002E2E2E5265D9
:10090800766572736520746F2025342E6400204D3F
:100918004F5645204572726F7200202E2E2E20539E
:1009280061766500202E2E2E2045646974002042D1
:10093800617365202025332E64202D2030782558BA
:1009480020200020536C696465204E756D626572C5
:1009580020256420002056616C75653A20256420A6
:1009680073202000204379636C653A202564207346
:1009780020200020456E61626C6564200020446977
:100988007361626C6564002056616C75653A202558
:1009980064205B25255D20200020466F72776172F8
:1009A80064202000204261636B77617264730020C9
:1009B8004C4F4720202D202025322E640020436FE5
:1009C8006E6669726D2052454C4F4144202E2E2E82
:1009D80000202E2E2E204C6F616465640020457225
:1009E8006173652043616C6962726174696F6E201E
:1009F8003F00202E2E2E2045726173656400204131
:100A0800646A75737420506F736974696F6E00201F
:100A1800536C6964652025322E6420446576202550
:100A2800322E642000205361766520536574746902
:100A38006E6773202E2E2E20200020436F6E66696D
:100A4800726D20434D44202E2E2E002053656C6578
:100A5800637420536C69646520312021210020567D
:100A6800616C75653A202564205B312F3130206D2B
:100A78006D5D20200020436F6E6669726D2054659D
:100A88007374202E2E2E00205344785020434F4D4F
:100A98004D206572726F72200020534478502043B5
:100AA8004F4D4D2070617373656400204D4F56455E
:100AB8004D454E54207061737365642000204D4F7E
:100AC80056454D454E54206572726F7220200020A5
:100AD8004465766963652046554E4354494F4E2018
:100AE8004F4B20200020446576696365204D414CBA
:100AF80046554E4354494F4E202000536F6674208C
:100B08005265736574202E2E2E00202E2E2E205016
:100B18006C65617365205761697400202E2E2E2044
:100B280053656C656374202020202020202020003D
:100B3800202E2E2E2045646974202000202E2E2E73
:100B48002043616E63656C20496E70757400202EB9
:100B58002E2E2053656C65637400534C4944452020
:100B68005649455720204250202F31320076657271
:100B780073696F6E20322E35370050454741535503
:100B8800532039382E2E2E303100205344785020EF
:100B9800434F4D4D206572726F7200494E49542083
:100BA8006279706173736564002573202D20253286
:100BB8002E64202F2025322E642000257300205417
:100BC800696D65206C6566743A2025332E64202093
:100BD80020200020416E616C6F67205B25255D2019
:100BE80025322E642025322E642020002041757481
:100BF8006F205363726F6C6C696E670020446D7868
:100C08002025332E64202D2025332E642025332ED5
:100C1800642020000000000000000BDD000017B970
:100C28000000239600002F7300003B4F0000472C64
:100C38000000530900005EE500006AC20000769FCC
:100C48000000827C00008E58205072696D617279B4
:100C580020636F6E74726F6C2020000020536571E2
:100C680075656E7469616C206163636573730000F8
:100C78002052616E646F6D20416363657373202039
:100C880020200000204175746F2054696D65722022
:100C98002020202020200000205363726F6C6C6994
:100CA8006E67202020202020202000002053696E1D
:100CB800676C65202020202020202020000020555F
:100CC8006E692D446972656374202020202000001D
:100CD8002042692D446972656374202020202020F9
:100CE800000020556E692D44697265637420496E51
:100CF800742E00002042692D44697265637420498E
:100D08006E742E2000004F7065726174696F6E20DA
:100D18006D6F646520200000444D58206164647242
:100D280065737320202020200000536C69646520BF
:100D38004E756D6265722020202000004578706F26
:100D4800737572652074696D652020200000466106
:100D580064696E672074696D65202020202000007A
:100D68004175746F54696D6572204D6F64652020FC
:100D780000005368757474657220436F6E74726FE7
:100D88006C2000005363726F6C6C2073706565642F
:100D98002020202000005363726F6C6C20646972FD
:100DA800656374696F6E000041636F75737469637E
:100DB8002062656570202020000052656C6F6164B8
:100DC8002064656661756C747320000043616C690A
:100DD80062726174696F6E202020202000004265D5
:100DE8006C7420636F7272656374696F6E200000A3
:100DF8004572726F7220636F646520202020202066
:100E08000000446961676E6F737469637320202002
:100E1800200000005072696D61727920005365717D
:100E280075656E63650052616E646F6D20200054B5
:100E3800696D6572202020005363726F6C6C2020EE
:100E48000020204E6F20726563657074696F6E00B4
:100E58004E6F2044494D4D45522064617461002015
:100E68002020446D782064617461204F4B0013206A
:0E0E78002D394653606C7986939FACB9C6D273
:1033E300044C00401454C110C112C111C18FC11348
:0733F300C10EC114015E00D0
:10000300E4FDEF4E6018EF1F70011E7C66EC600884
:0E0013001CEDF5F0A4FD80F5D2AED2BE80E467
:0100210022BC
:0C343500EF60091F7E15EE60F71E80FAA4
:013441002268
:02348C0000221C
:10324D00AD07AC06300825D2ECC2EEED25E0FDEC65
:10325D0033FCED4C6012ED1D70011C7F05123435F1
:0D326D00B2EBD2AED2BE80EAC2ECC2EB22C0
:102DEB00AB07AA06ED14601D14602514602624039E
:102DFB00702D7D64EBAE027802CEC313CE13D8F9DF
:102E0B00FBAA06802B7D32EAC313FAEB13FB80205F
:102E1B007D19801C7D0AEB25E0FBEA33FA80117DDE
:102E2B0005EBAE027802C333CE33CED8F9FBAA063C
:102E3B00D2ECC2EEEB4A6012EB1B70011AAF05121B
:0F2E4B003435B2EBD2AED2BE80EAC2ECC2EB227B
:0C345C00D2ED0000C2ED7F0112343522D9
:1032CF007FFFAEE843E80FC2EFC2ECD2EED2ED00C3
:1032DF0030EB0AEF60071FD2AED2BE80F3C2ED0013
:0832EF008EE8EF6002D322C358
:0132F70022B4
:10002600AD07C2EC1232CFD2ED53E8F0EDC4540F57
:10003600540F42E812345CD2ED53E8F0ED540F420F
:05004600E812345C2209
:0D344200C2EEC2EFC2EC430780120026224A
:10290200C2EEC2EFC2EDC2EC3003097F147E0012A8
:10291200000380077F017E00120003D2ED53E8F02E
:1029220043E80312345C7F057E00120003D2ED53AC
:10293200E8F043E80312345C7F017E00120003D208
:10294200ED53E8F043E80312345C7F017E0012008D
:1029520003D2ED53E8F043E80212345C7F017E00BB
:102962001200037F281200267F0C1200267F061217
:1029720000267F011200267F021200267F027E00BF
:04298200120003221A
:1033FB007F011200267F027E001200037F02120063
:07340B0026E4FF1234422207
:0A347300D2EFC2EE120026C2EF22D3
:10318E008B3A8A3B893CD2EFC2EEAB3AAA3BA93CC2
:10319E001212D8FF60171200267401253CF53CE48C
:1031AE00353BF53B7F017E0012000380DDC2EF222E
:0431BE00AC07AB05AA
:1031C200744B2CF8E6FF123442E4FAC3EB6480F845
:1031D200EA648098500C7F20123473D2AED2BE0AB9
:0B31E20080E9744B2CF8E6FF12344229
:0131ED0022BF
:10342400300304C2968002D2967F017E001200030C
:013434002275
:05347D00D2F8D2F92293
:062986008B3E8A3F8940F0
:10298C00C2F812348CC2F9EF25E054FEFFE4FEEFDE
:10299C0025E0FF92F8D2F9C2F90EBE08F2D2F8D2B5
:1029AC00F9A2F8B3920AC2F9200902D20A300A41FC
:1029BC00E541603DAB3EAA3FA9401212D8FFE4FEB0
:1029CC00EF25E0FF92F8D2F9C2F90EBE08F2D2F868
:1029DC00D2F9A2F8B3920AC2F974012540F540E489
:1029EC00353FF53F1541200902D20AD2AED2BE8046
:0C29FC00BCC2F8D2F912348CD2F8A20A46
:012A080022AB
:0627F4008B3D8A3E893F87
:1027FA00E4FE7D80C2F812348CC2F9EF25E0440170
:10280A00FFE4FCEF25E0FF92F8D2F9C2F90CBC080C
:10281A00F2D2F8D2F9A2F8B39208C2F9300848E520
:10282A00406044E4FFFCD2F930F803ED4207C2F9F4
:10283A00EDC313FD0CBC08EEAB3DAA3EA93FEF1257
:10284A0012F11540E5406004C2F88002D2F8D2F9CC
:10285A0012348CC2F97401253FF53FE4353EF53E4A
:10286A000ED2AED2BE80B5C2F8D2F912348CD2F8EA
:02287A00AF06A7
:01287C002239
:10315D00C208753C0A7866A60708A60520081FE573
:10316D003C601B7F017E001200037B007A007966B4
:10317D00754102D2097F50122986920880DEA2087D
:01318D00221F
:1030EB00C205752E0A7866A607ECFF3395E0EF084C
:1030FB00F6ED08F620051FE52E601B7F017E001202
:10310B0000037B007A007966754103D2097F501268
:08311B002986920580DEA20561
:013123002289
:103345007866A6077B007A007966754101D2097F08
:10335500501229867B007A0079667540017F5012EC
:0533650027F4E6FF2241
:022F90008F357B
:102F92007866A6357B007A007966754101D2097F91
:102FA200501229867B007A0079667540017F5012A3
:102FB20027F4E6F536E53504F67B007A0079667586
:102FC2004101D2097F501229867B007A0079667509
:102FD20040017F501227F4E536FEE67C002400FF14
:032FE200EC3EFEC4
:012FE50022C9
:05348200D2B4D2B52216
:02312400AC07F6
:10312600ED6024A804E6FB7A08EA6012EB25E0FBD2
:103136001A92B4C2B5D2B57F0112343580EB0C1D9C
:103146007F0112343580D9D2B4D2B57F0512343519
:0631560030B402C322D3D5
:01315C002250
:102FE6007B7820940BA20692087F0A7E0012324D4F
:102FF60043E80FD2EED2ECE5E8540FFA30051B2079
:103006009418EB600A7F0A7E001200031B80F0D240
:10301600087F0A7E0012324D80E5C2EEC2ECC2C1C4
:06302600C210D2B9AF0296
:01302C002281
:10336A007B78209418EB600A7F0A7E001200031B08
:10337A0080F0D2087F0A7E0012324D80E5C2C1C2B7
:03338A0010D2B9A5
:01338D00221D
:0D344F003094097F017E0012000380F422FA
:02302D008F3AD8
:10302F007F301233458F3BE53B2431FFAD3A1231F0
:10303F005D053BE53BC3940550028001C34003E4AB
:10304F00F53BAD3B7F3012315DE4FBD2087F1E7E36
:0F305F000012324D7FC87E001200030BBB06EC3F
:01306E00223F
:102F2B007F301233458F2C152CE4F52DE52CC394F3
:102F3B000550028001C34003752C04E52C2431FF9E
:102F4B00123345742E252DF8A607152C052DE52DCE
:102F5B00C3940540D7E4F52DE52D75F003A4246645
:102F6B00F9E4FAFB753BFF753C08753D08742E259B
:102F7B002DF8E6753E00F53F120EE2052DE52DC34B
:042F8B00940540D495
:012F8F00221F
:10338E00E4FD7F3012315DE4F52CE52C2431FF7D18
:0D339E00FF12315D052CE52CC3940540EDB8
:0133AB0022FF
:10327A001233FB7F401234427B007A0079661231A6
:10328A008E7F141234427BFF7A08790F12318E7FB7
:0B329A00F212302DD2AED2BE80FA221C
:1033AC00ED14FEEED39400400EEF2E14F8E6FDEF74
:0B33BC002EF8A6051E80ECA807A60353
:0133C70022E3
:10331F00E4F510F511FEEEC39D5010A807E6251138
:10332F00F511E43510F5100E0F80EBED7C00AE10AB
:05333F00AF1112136A3A
:013344002266
:1030B100ED14FEC3EE64809480402E7D01D3EE6456
:1030C10080F8ED648098501EEF2DF8E6FCE814F8C6
:1030D100E6FBD39C400DA903EF2D14F8A604EF2DB8
:0930E100F8A6010D80D71E80CA7B
:0130EA0022C3
:1031EE001233FB7F401234427BFF7A08791E123174
:1031FE008E7F141234427BFF7A08793212318E7F21
:10320E00F112302DD2087FD07E0712324D80FE2271
:04287D008F2D8D2EE0
:10288100752F05753005C204786676800876810853
:1028910076827966E7182624827869F6200443E572
:1028A10030603FE52DC313452EFF7B007A0079662A
:1028B100754104D2091229864011E52F600DD20815
:1028C1007F0A7E0012324D152F80D87F04123435D5
:1028D10020F904D20480077F327E001200031530F4
:1028E10080BA7FC87E00120003E52F6006E53060E4
:1028F10002D322D2087FD07E0712324D1231EEC3AD
:0129010022B3
:0825BF008F328D338A348B3515
:1025C700753605753705C20478667690E534FF33AE
:1025D70095E0EF08F6AF35E53508F6FF7966E718B9
:1025E700262F7869F6200443E537603FE532C313A9
:1025F7004533FF7B007A007966754104D2091229B9
:10260700864011E536600DD2087F0A7E0012324DF2
:10261700153680D87F0412343520F904D204800798
:102627007F327E00120003153780BA7FC87E001202
:102637000003E5366009E5376005AE34AF35221291
:0626470031EE7EFF7FFF73
:01264D00226A
:042B85008F2F8D30D1
:102B8900753305753405C205786676A008A603086D
:102B9900A6327966E7182625327869F6200543E5D5
:102BA90034603FE52FC3134530FF7B007A00796617
:102BB900754104D2091229864011E533600DD20806
:102BC9007F0A7E0012324D153380D87F04123435C6
:102BD90020F904D20580077F327E001200031534E4
:102BE90080BA7F647E00120003E5336006E5346035
:072BF90002D3221231EEC3EA
:012C000022B1
:04252C008F2A8D2B3A
:10253000753005753105C203786676C0AE02AF030B
:102540007C007D6412136A7867A607AE2EAF2F7CDD
:10255000007D6412136A7868EFF67966E718262F13
:102560007869F6200343E531603FE52AC313452B24
:10257000FF7B007A007966754104D20912298640F2
:1025800011E530600DD2087F0A7E0012324D153001
:1025900080D87F0412343520F904D20380077F32BB
:1025A0007E00120003153180BA7F647E00120003A2
:0E25B000E5306006E5316002D3221231EEC341
:0125BE0022FA
:042A09008F2A8D2B58
:102A0D00752F05753005C203786676B008A603E507
:102A1D002DC313E52E13FF08F67966E718262F78D8
:102A2D0069F6200343E530603FE52AC313452BFFCC
:102A3D007B007A007966754104D20912298640110E
:102A4D00E52F600DD2087F0A7E0012324D152F80C2
:102A5D00D87F0412343520F904D20380077F327EEB
:102A6D0000120003153080BA7F647E00120003E56A
:0D2A7D002F6006E5306002D3221231EEC357
:012A8A002229
:042C01008F2A8D2B5E
:102C0500752E05752F05C203786676D008A60308CC
:102C1500A62D7966E71826252D7869F6200343E564
:102C25002F603FE52AC313452BFF7B007A007966A9
:102C3500754104D2091229864011E52E600DD2088E
:102C45007F0A7E0012324D152E80D87F041234354E
:102C550020F904D20380077F327E00120003152F6E
:102C650080BA7F647E00120003E52E6006E52F60C2
:072C750002D3221231EEC36D
:012C7C002235
:042A8B008F2A8D2BD6
:102A8F00752C05752D05C203786676E0EA08F6AF5A
:102A9F0003EB08F67966E718262F7869F6200343CB
:102AAF00E52D603FE52AC313452BFF7B007A0079A4
:102ABF0066754104D2091229864011E52C600DD2AA
:102ACF00087F0A7E0012324D152C80D87F041234F5
:102ADF003520F904D20380077F327E0012000315E0
:102AEF002D80BA7F647E00120003E52C6006E52D71
:082AFF006002D3221231EEC384
:012B070022AB
:042B08008F2F8D304E
:102B0C00753105753205C20578667620300404E609
:102B1C004401F6786776AA0876BB7966E71826240E
:102B2C00BB7869F6200543E532603FE52FC31345BA
:102B3C0030FF7B007A007966754104D20912298630
:102B4C004011E531600DD2087F0A7E0012324D151E
:102B5C003180D87F0412343520F904D20580077FE8
:102B6C00327E00120003153280BAE5316006E53280
:082B7C006002D3221231EEC306
:012B8400222E
:0826DC008F328D338A348B35F7
:1026E400753805753905C205D3E5359537E5349553
:1026F40036400685363485373578667638E53408CD
:10270400F6AF35E53508F6FF7966E718262F7869C0
:10271400F6200543E539603FE532C3134533FF7BBB
:10272400007A007966754104D2091229864011E5C0
:1027340038600DD2087F0A7E0012324D153880D8D9
:102744007F0412343520F904D20580077F327E00DD
:10275400120003153980BAE5396005AE34AF35226D
:032764001231EE41
:01276700224F
:041BA6008F2E8D2FC2
:101BAA00753605753705C207E5332BE5323AC39416
:101BBA00005009C3E49BF533E49AF532E5332BFF71
:101BCA00E5323AFED3EF9535EE9534400AE5359B7A
:101BDA00F533E5349AF532D3E5339400E53264807F
:101BEA009480400878667611D20680067866761068
:101BFA00C2063005067866E64404F6AF33AE321202
:101C0A0034128E328F33E53345327003021C9AE563
:101C1A0032FF3395E0EF7867F6AF33E53308F6FF26
:101C2A007966E718262F7869F6200743E537603F7B
:101C3A00E52EC313452FFF7B007A007966754104B0
:101C4A00D2091229864011E536600DD2087F0A7E34
:101C5A000012324D153680D87F0412343520F9042B
:101C6A00D20780077F327E00120003153780BAE55B
:101C7A003760197F037E00120003300605AE32AFCB
:101C8A003322C3E49533FFE49532FE221231EE2269
:041C9A007E007F0049
:011C9E002223
:10192F00300450AD5BAC5A7F101230EBAD577F23B4
:10193F0012315DAD507F2012315DAD517F241231D8
:10194F005DAD527F2512315DAD537F2212315DADFA
:10195F00587F2612315DAD547F2712315DAD597F0F
:10196F002912315DAD567F2812315DAD557F2112A1
:10197F00315D227F10122F908E5A8F5BC3E55B94DF
:10198F0001E55A9400400BD3E55B94FCE55A9401B2
:10199F004006755A00755B017F231233458F57D36D
:1019AF00E557648094845009C3E557648094805050
:1019BF0003E4F5577F201233458F50E550D3940C35
:1019CF005007E550C39401500375500C7F24123318
:1019DF00458F51E551D394965007E551C39401506B
:1019EF000375510A7F251233458F52E552D3943C2C
:1019FF005007E552C3940150037552057F261233E9
:101A0F00458F58D3E558648094855009C3E55864D1
:101A1F0080948150037558027F271233458F54E508
:101A2F0054D394645007E554C39401500375545034
:101A3F007F291233458F59D3E5596480948A500911
:101A4F00C3E559648094765003E4F5597F28123327
:101A5F00458F567F211233458F557F221233458F85
:021A6F00532200
:0B34680075988075A910C298C29922C7
:10321E0053D8F8EF540742D8C2DBE4FB75DA8020AE
:10322E00DCFD74662BF8A6D97F037E001200030B1B
:0E323E00BB03E97F667D031230B17867E6FFBF
:01324C00225F
:1033C800D291EF25E0540744017866F608A6057FF8
:0B33D800667D02123124C291D29122C6
:041E77008F328D33E6
:101E7B007F54123442753BFF753C08753D407B0027
:101E8B007A007966120EE27B007A00796612318E47
:101E9B00E532601FFF3395E0FE7C007D0E121303CD
:101EAB007C637D9CCFCDCFCECCCE12136A8E348F7C
:101EBB0035800675346375359CE533249B604D0482
:101ECB006003021F5EE4F536F537AE36AF377C00A4
:101EDB007D6412136AAD07E4FF1233C87F477E009F
:101EEB00120003E5352537F537E5343536F536C3BE
:101EFB00E537949CE536648094E340CE7DFFE4FFA8
:101F0B001233C87D147F041231BEC322753663753C
:101F1B00379CAE36AF377C007D6412136AAD07E495
:101F2B00FF1233C87F477E00120003C3E537953598
:101F3B00F537E5369534F536D3E5379400E5366459
:101F4B0080948050CDE4FDFF1233C87D147F0412C2
:031F5B0031BED3C1
:011F5E002260
:101C9F007F54123442753BFF753C08753D557B00F0
:101CAF007A007966120EE27B007A00796612318E25
:101CBF0075323CE4FBFD7FB0122B8530B229C20494
:101CCF00E4FD7FB0122B08752D4E752E2030B21704
:101CDF00E52E452D60117F017E00120003E52E15C4
:101CEF002E7002152D80E6D204E4FD7FB0122B0872
:101CFF00752D4E752E2020B217E52E452D60117FC4
:101D0F00017E00120003E52E152E7002152D80E6C0
:101D1F00C2F87F017E00120003D2F87F647E0012AA
:101D2F00000375368F7537247B037A00E4FD7FB08F
:101D3F001226DC7FFA7E00120003E55425E024050D
:101D4F00F532E4FBFD7FB0122B85D20F7B057A00B5
:101D5F00E4FD7FB01225BFC20EE52E452D70157F15
:101D6F00541234427BFF7A08796A12318E7F121235
:0B1D7F00302D80FE7D147F041231BE69
:011D8A002236
:10306F007532A0E4FBFD7FB0122B85752D00752EF8
:10307F00FA7B24E4FD7FB0122A09752E05752F14F3
:10308F007B587A02E4FD7FB012252CE4F52D7B648A
:10309F00FD7FB0122C017BC07A8EE4FD7FB0122A27
:0230AF008B2272
:10264E007BFF7A08797D12318E7F401234427BFFF8
:10265E007A08798D12318E20B25D7BC07A8EE4FDC0
:10266E007FB01225BFC204E4FD7FB0122B087FE8B5
:10267E007E031200037B207A4E20B212EB4A600ECC
:10268E007F057E00120003EB1B70011A80EBC2F86F
:10269E007F017E00120003D2F8EB4A701A7F1012EF
:1026AE00302D753BFF753C08753DA07B007A007997
:1026BE0066120EE212327A7F141234427BFF7A08CF
:0D26CE0079B212318E121C9F1233FB7F0176
:0126DB0022DC
:022494008F3285
:102496001532E532700302252725E02440FF122F6E
:1024A600908E338F34E53225E025E0241CF582E456
:1024B600340CF5831213B1EF241EFBE43EFAE43D1F
:1024C600F9E43CF8AE33AF34E4FCFDC31213A0408C
:1024D6002FE53225E025E0241CF582E4340CF58353
:1024E6001213B1EF24E2FBEE34FFFAED34FFF9EC00
:1024F60034FFF8AE33AF34E4FCFDD31213A0401C16
:102506007D037FC87E00122DEBE53225E025E02411
:102516001CF582E4340CF5831213B122AE33AF34CA
:05252600227E007F0091
:01252B00228D
:061450008F2DAB05AA047C
:10145600852D2E752F05E55EB52D01227F141234DC
:1014660042EB4A600DE55360097D65AF52121E7767
:101476009214E52DB4011AE550C3132401FFE43399
:10148600FED3E55E9FEE6480F87480984003752D68
:101496000D752F0520FF03021608E52DD395504044
:1014A6005C7BFF7A0879C612318E300F277F0D12CA
:1014B6002494AD59ED3395E0FCEF2DFFEE3CCF249F
:1014C60005FBE43FFA75368F753724E4FD7FB012CD
:1014D60026DC801F7F0D122494AD59ED3395E0FC78
:1014E600EF2DFBEE3CFA75368F753724E4FD7FB0A1
:1014F6001226DCB20ED20F752E010215F8E52DC3A9
:1015060094015068300F157F0D122494EF2405FBCB
:10151600E43EFAE4FD7FB01225BF80107F0D122451
:1015260094AA06AB07E4FD7FB01225BF7BFF7A08BD
:1015360079DB12318EE557B4030FE558B4040AE59A
:101546005020E00514F52D800385502DAF2D122473
:1015560094AA06AB0775368E7537C0E4FD7FB012C8
:1015660026DCB20EC20F852D2E0215F8E52DD39579
:101576005E4042AF2D1224948E308F31EF2405FB4E
:10158600E43EFA75368E7537C0E4FD7FB01226DC70
:10159600D20F753BFF753C08753DF085303E8531B1
:1015A6003F7B007A007966120EE27B007A0079664C
:1015B60012318E803DAF2D122494AA068A30AB07D5
:1015C6008B3175368E7537C0E4FD7FB01226DCC2CE
:1015D6000F753BFF753C09753D0385303E85313FF0
:1015E6007B007A007966120EE27B007A0079661239
:1015F600318E7F647E00120003152FE52F600302F3
:10160600149AE52F70157F541234427BFF7A0979BC
:0F1616001612318E7F1112302D80FED213AF2E9F
:0116250022A2
:03004B00023487F5
:05348700D210C2B932B1
:03002300022E5A50
:102E5A00C0E0C0D075D008309A41301256301118EF
:102E6A00C211E5996005755F018048755F02E55DED
:102E7A00155D7002155C803BE55D455C600AE55DA9
:102E8A00155D7002155C802B74612560F8A699E5C2
:102E9A006060041560801CC2128018E599700F8565
:102EAA005A5C855B5D756004D211D2128005C2122C
:0A2EBA00755F0AC298D0D0D0E03254
:1020180085572BC203D205A2039206122FE6EF645E
:1020280002607BBF040E1557C3E557648094805047
:1020380003E4F557BF080E0557D3E5576480948429
:102048004003755704EF640170287F541234427BB3
:10205800FF7A09792212318ED20412192F7FE87E75
:10206800031200037F541234427BFF7A09792C1241
:10207800318E7F40123442AF57EF3395E0FE7C003B
:102088007D1412130374502FF9740C3EFA7BFF125F
:10209800318EE55524FF920312344F02201DE52BA3
:1020A800B40408E5576404600280FEE52B6403600D
:1020B80010E557B4030B7D017C007F011214508F8B
:0120C8005EB9
:0120C90022F4
:101F5F00C205C206122FE6EF6402700302200ABF09
:101F6F000417055BE55B7002055AD394FCE55A94A0
:101F7F00014006755A00755B01BF0819E55B155BDB
:101F8F007002155AC3E55B9401E55A94005006752B
:101F9F005A01755BFCEF640170287F541234427B49
:101FAF00FF7A09792212318ED20412192F7FE87E1F
:101FBF00031200037F541234427BFF7A09792C12EB
:101FCF00318E7F40123442753BFF753C09753D36AB
:101FDF00855A3E855B3F855A40855B417B007A0081
:101FEF007966120EE27B007A00796612318E7FC815
:101FFF007E0012000312344F021F5FE55524FF923B
:08200F00087F0A7E0012324D29
:0120170022A6
:1021750085502BC205C206122FE6EF6402700302DA
:102185002205BF040C0550E550D3940C400375504F
:102195000CBF080C1550E550C39401500375500150
:1021A500EF640170287F541234427BFF7A0979224B
:1021B50012318ED20412192F7FE87E031200037F9D
:1021C500541234427BFF7A09792C12318E7F4012EA
:1021D5003442753BFF753C09753D4B753E00855096
:1021E5003F7B007A007966120EE27B007A00796601
:1021F50012318E7FC87E0012000312344F022178FF
:10220500E55524FF92087F0A7E0012324DE55065A0
:052215002B600280FEB9
:01221A0022A1
:10235E00C205C206122FE6EF640270030223EBBF22
:10236E00040C0551E551D394964003755101BF08F5
:10237E000C1551E551C394015003755196EF64014C
:10238E0070287F541234427BFF7A09792212318EE3
:10239E00D20412192F7FE87E031200037F541234E9
:1023AE00427BFF7A09792C12318E7F4012344275AE
:1023BE003BFF753C09753D5D753E0085513F7B00C9
:1023CE007A007966120EE27B007A00796612318EFF
:1023DE007FC87E0012000312344F02235EE555249F
:0A23EE00FF92087F0A7E0012324DB4
:0123F80022C2
:1023F900C205C206122FE6EF64027003022486BFEB
:10240900040C0552E552D3943C4003755201BF08B0
:102419000C1552E552C39401500375523CEF640107
:1024290070287F541234427BFF7A09792212318E47
:10243900D20412192F7FE87E031200037F5412344D
:10244900427BFF7A09792C12318E7F401234427512
:102459003BFF753C09753D6C753E0085523F7B001D
:102469007A007966120EE27B007A00796612318E63
:102479007FC87E0012000312344F0223F9E5552468
:0A248900FF92087F0A7E0012324D18
:012493002226
:102C7D00C203D205A2039206122FE6EF6402606929
:102C8D00EF64046003BF080CE55370047E018002FD
:102C9D007E008E53EF640170287F541234427BFF07
:102CAD007A09792212318ED20412192F7FE87E0310
:102CBD001200037F541234427BFF7A09792C1231B2
:102CCD008E7F40123442E553600B7BFF7A09797B8E
:102CDD0012318E80097BFF7A09798512318EE55587
:092CED0024FF920312344F808988
:012CF60022BB
:1022BE0085582BC203D205A2039206122FE6EF64B5
:1022CE0002607BBF040E1558C3E55864809481509C
:1022DE0003755801BF080E0558D3E55864809485E0
:1022EE004003755805EF640170287F541234427B09
:1022FE00FF7A09792212318ED20412192F7FE87ECD
:10230E00031200037F541234427BFF7A09792C1298
:10231E00318E7F40123442AF58EF3395E0FE7C0091
:10232E007D1212130374A22FF9740C3EFA7BFF1266
:10233E00318EE55524FF920312344F0222C3E52B52
:0F234E006558600B7D017C007F011214508F5E7B
:01235D00225D
:1020CA00C205C206122FE6EF64027003022157BF4F
:1020DA00040C0554E554D394644003755401BF08B5
:1020EA000C1554E554C394015003755464EF64010C
:1020FA0070287F541234427BFF7A09792212318E7A
:10210A00D20412192F7FE87E031200037F5412347F
:10211A00427BFF7A09792C12318E7F401234427544
:10212A003BFF753C09753D8F753E0085543F7B002A
:10213A007A007966120EE27B007A00796612318E95
:10214A007FC87E0012000312344F0220CAE55425CC
:10215A00E02405F532E4FBFD7FB0122B85E555241A
:0A216A00FF92087F0A7E0012324D3A
:012174002248
:102CF700C203D205A2039206122FE6EF64026069AF
:102D0700EF64046003BF080CE55670047E0180027F
:102D17007E008E56EF640170287F541234427BFF89
:102D27007A09792212318ED20412192F7FE87E0395
:102D37001200037F541234427BFF7A09792C123137
:102D47008E7F40123442E556600B7BFF7A0979A1EA
:102D570012318E80097BFF7A0979AC12318EE555E5
:092D670024FF920312344F80890D
:012D70002240
:102EC400C2037D147F041231BED205A203920612FE
:102ED4002FE68F2BEF640260467F401234427F302E
:102EE400123345753E008F3F753BFF753C09753DB8
:102EF400B77B007A007966120EE27B007A0079666D
:102F040012318E7F14123442122F2B7B007A0079F7
:102F14006612318EE55524FF920312344F80AA7D48
:062F2400147F031231BE10
:012F2A002284
:102D7100C203D205A2039206122FE6EF6402606934
:102D8100EF64046003BF080CE55570047E01800206
:102D91007E008E55EF640170287F541234427BFF10
:102DA1007A09792212318ED20412192F7FE87E031B
:102DB1001200037F541234427BFF7A09792C1231BD
:102DC1008E7F40123442E555600B7BFF7A09797B97
:102DD10012318E80097BFF7A09798512318EE55592
:092DE10024FF920312344F808993
:012DEA0022C6
:101D8B00C2037F401234427BFF7A0979C512318E30
:101D9B00E55524FF920312344FD205A2039206128B
:101DAB002FE6EF64016003021E76F557F55A755B5B
:101DBB000175500C75510A755205F553755802751E
:101DCB00545075560175550112338E7F541234429F
:101DDB007BFF7A0979D912318ED20412192F7FE841
:101DEB007E031200037D147F041231BE7F40123438
:101DFB00427BFF7A0979E512318E12344FD205A25C
:101E0B00039206122FE6EF64017060F52BD3E52BDE
:101E1B006480948C4003D38001C34033E52B25E0D1
:101E2B002440FFC007AF2BEF3395E0FEEF7802C3E2
:101E3B0033CE33CED8F9241CF582740C3EF58312C5
:101E4B0013B1AD07AC06D0071230EB052B80BE7F6C
:101E5B00541234427BFF7A0979FA12318E7FE87E75
:0B1E6B00031200037D147F041231BE3F
:011E76002249
:10162600C203C204E55E640160030217B4D205A2D8
:10163600039206122FE68F2BEF640270030217C97E
:10164600E55E640C70030217C9E52B6401600302B2
:10165600179A7F401234427BFF7A0A790612318E3E
:10166600755450E55425E02419F532E4FBFD7FB0AE
:10167600122B85755E02E55ED3940C4003D3800180
:10168600C35003021798E55E25E025E02418F5828D
:10169600E4340CF5831213B1EF24E7FBEE34FFFAC2
:1016A60075368E7537C0E4FD7FB01226DC7FFA7E74
:1016B60000120003752DC220FF0A7F327E00120041
:1016C60003D52DF3E52D700280FE752CE27F5412B2
:1016D6003442753BFF753C0A753D17753E00855EC5
:1016E6003FAF2CEF3395E0F5408F417B007A0079D0
:1016F60066120EE27B007A00796612318E12344F42
:10170600D205A2039206122FE68F2BE52B640470F6
:101716002D052CF53275330175348E7535C0C2052D
:10172600FBFAFD7FB0121BA6752DC220FF0A7F0AA9
:101736007E00120003D52DF3E52D700280FEC3E571
:101746002C6480949E5006E52B640170807F5412B1
:1017560034427BFF7A0A792D12318EE55E25E0252B
:10176600E02418F582E4340CF5831213B1AD2CEDA8
:101776003395E0FCEF2DFDEE3CFCE55E14FF25E025
:101786002440FF1230EB7FE87E03120003055E0261
:10179600167C80FE7F401234427BFF7A0A79421221
:1017A600318EE55524FF920312344F0216337F40E3
:1017B6001234427BFF7A0A795312318E7FE87E0318
:0317C6001200030B
:0117C90022FD
:10221B00C205C206122FE6EF640270030222B0BFA2
:10222B00040E0559D3E5596480948A400375590A05
:10223B00BF080E1559C3E559648094765003755940
:10224B00F6EF640170287F541234427BFF7A0979D0
:10225B002212318ED20412192F7FE87E0312000353
:10226B007F541234427BFF7A09792C12318E7F40D6
:10227B00123442753BFF753C0A753D66AF59EF331F
:10228B0095E0F53E8F3F7B007A007966120EE27B7C
:10229B00007A00796612318E7FC87E00120003121D
:1022AB00344F02221BE55524FF92087F0A7E001251
:0222BB00324DA2
:0122BD0022FE
:101A7100C2037F401234427BFF7A0A797D12318E94
:101A810012344FD205D206122FE6EF640160030231
:101A91001BA57F40123442E4FD7FB012287D401621
:101AA100753BFF753C0A753D8F7B007A00796612A4
:101AB1000EE2D2038012753BFF753C0A753DA17B96
:101AC100007A007966120EE27B007A0079661231A3
:101AD1008E7FD07E071200037532A0E4FBFD7FB03C
:101AE100122B85E4FDFC7F011214508F5E7FDC7E9A
:101AF10005120003752B0B752CB820FF1A7F0A7E87
:101B010000120003E52C152C7002152BD3E52C9443
:101B110000E52B940050E37D147F031231BE7F401A
:101B2100123442E52C452B6014753BFF753C0A7558
:101B31003DB37B007A007966120EE28014753BFF9B
:101B4100753C0A753DC57B007A007966120EE2D2BA
:101B5100037B007A00796612318E7FD07E071200F6
:101B610003200317121C9F753BFF753C0A753DD777
:101B71007B007A007966120EE28012753BFF753C9C
:101B81000A753DED7B007A007966120EE27F401204
:101B910034427B007A00796612318E7F887E13127F
:041BA100000380FEBF
:011BA500221D
:1032A5001233FBE4FF1234427BFF7A0B79031231B0
:1032B5008E7F401234427BFF7A0B791212318E12C7
:0A32C500336A7FF012302D80FE22E4
:1017CA00E4F52A1233FBE4FF123442AF2AEF3395D1
:1017DA00E0FE7C007D12121303740E2FF9740D3E85
:1017EA00FA7BFF12318E7F541234427BFF7A0B79D7
:1017FA002312318E12336A12344FD205E55524FF73
:10180A009206122FE6EF64027003021927BF040A38
:10181A00052AE52AB40F03E4F52ABF080E152AC3E0
:10182A00E52A648094805003752A0EEF64016003F0
:10183A000219017F541234427BFF7A0B7938123134
:10184A008EE52AB40F0040030218D490185CF828D9
:10185A00287302188902188E02189302189802181F
:10186A009D0218A20218A70218AC0218B10218B6F3
:10187A000218BB0218C00218C50218CA0218CF12F1
:10188A002018805B121F5F80561221758051122327
:10189A005E804C1223F980471222BE8042122C7DB0
:1018AA00803D1220CA8038122CF78033122D7180A5
:1018BA002E121D8B8029121626802412221B801FAD
:1018CA00122EC4801A121A7180157F401234427B7C
:1018DA00FF7A0B794412318E7FE87E031200037D72
:1018EA00147F021231BE7F541234427BFF7A0B7985
:1018FA005612318E12336AE4FF123442AF2AEF33A2
:10190A0095E0FE7C007D12121303740E2FF9740DFC
:10191A003EFA7BFF12318E12344F0218047D147F77
:04192A00041231BEB4
:01192E002296
:10004E00E4F5237524FA75251E7526FFD200D2011C
:10005E00D202F587F5D012347D123482123468D272
:10006E00BED297F55FC20412192F7E007F007D0568
:10007E007B007A0079611213C1D2B9C2CDD2AFD250
:10008E009CC298D2ACD203122902E4FF1234427BF6
:10009E00FF7A0B796212318E7F471234427BFF7AE0
:1000AE000B797512318E7F591234427BFF7A0B79A0
:1000BE008212318ED2031234247FB87E0B120003CB
:1000CE001233FB7E007F067D007B007A00797F1263
:1000DE0013C1E4F527E4FDAF271233C87F0A7E0073
:1000EE001200030527E527C3940240E9E4FD7FB023
:1000FE0012287D4015753BFF753C0B753D927B00BC
:10010E007A007966120EE212327AD2087FC87E0029
:10011E0012324D12306FC205C206122FE6EF640383
:10012E00703F7F401234427BFF7A0B79A312318EDF
:10013E00E4F527D2087F647E0012324D7F647E0084
:10014E001200030527E527C3940A40E7E4FBFAFDF6
:10015E007FB01225BF755E017D147F021231BE8005
:10016E000512264E8F5EE55175F00AA485F028F52E
:10017E0029E557B403077DFFE4FF1233C8E5266077
:10018E00041526800B7526FFE4F525C203122902FD
:10019E00E4FF123442AF57EF3395E0FE7C007D0949
:1001AE00121303741C2FF9740E3E753EFFF53F8932
:1001BE0040753BFF753C0B753DB1754100855E4248
:1001CE007543008550447B007A007966120EE27BFF
:1001DE00007A00796612318E201003209437D203F4
:1001EE001234247524FAC205C206122FE68F23BFDD
:1001FE00030ED297D2087F0A7E0012324D1232A51C
:10020E00E523B40113D297D2087F0A7E0012324D35
:10021E001217CA8003E4F523E4F527E52775F003EA
:10022E00A4247FFFC3740495272461F8E6FB7D03A5
:10023E001233ACE52775F003A4247FF9E4FAFB78BA
:10024E00667C00FDFE7F031212B27F667D031230C4
:10025E00B17867E6FF74142527F8A6070527E5276A
:10026E00C3940240B6E52560041525803A7F5A12E4
:10027E003442E55F75F00FA42449F9740E35F0751C
:10028E003EFFF53F8940753BFF753C0B753DC37BCB
:10029E00007A007966120EE27B007A0079661231DE
:1002AE008E75251EE4F55FE4FF12321E7812A60746
:1002BE007F0112321E7813A607E557603F24FC70AB
:1002CE000302035C04600302036C7F40123442AEEF
:1002DE0028AF297C007D0A1213158E3E8F3F753B89
:1002EE00FF753C0B753DC67B007A007966120EE2F7
:1002FE007B007A00796612318E0203BE7F40123483
:10030E00427812E6FF7E007C007D641213037DFFAF
:10031E00121315AA06AB077813E6FF7E007C007D4C
:10032E00641213037DFF1213158E408F418A3E8B8C
:10033E003F753BFF753C0B753DDB7B007A007966A4
:10034E00120EE27B007A00796612318E80627F4057
:10035E001234427BFF7A0B79F412318E80527F4039
:10036E00123442AF657E007C007D641213037DFF64
:10037E00121315AA06AB07AF647E007C007D6412D3
:10038E0013037DFF1213158E428F438A408B4175E6
:10039E003BFF753C0C753D04855A3E855B3F7B00EB
:1003AE007A007966120EE27B007A00796612318E3F
:1003BE00E5571470030204F31470030205A01470C1
:1003CE00030206291470030207792404600302074E
:1003DE00897812E6FFD3943F4013EF9466500E08CF
:1003EE00E6FF943F4007EF94665002C200301303BD
:1003FE00020789E52324F8601724FC602224087084
:10040E0029E55E04FF7D017C001214508F5E801A78
:10041E00E55E14FF7D017C001214508F5E800B7D13
:10042E00017C007F011214508F5E30000302078999
:10043E007812E6C39434501508E6943F400FE55EFB
:10044E0004FF7D017C001214508F5ED2007812E6FC
:10045E00D3943F401508E69434500FE55E14FF7DAB
:10046E00017C001214508F5ED2007812E6C39434D1
:10047E00501408E6C39434500D7D017C007F0112A8
:10048E0014508F5ED2007812E6D394B4401508E66D
:10049E009466500FE55E04FF7D017C001214508FB0
:1004AE005ED2007812E6C39466501508E694B44006
:1004BE000FE55E14FF7D017C001214508F5ED2009A
:1004CE007812E6D394B4500302078908E6D394B4A5
:1004DE0050030207897D017C007F011214508F5E4C
:1004EE00D2000207897814E6C3944C500908E6C37B
:1004FE00944C5002C201301303020789E52324F8FD
:10050E00601624FC602024087026E55E04FFE4FDDE
:10051E00FC1214508F5E8018E55E14FFE4FDFC1291
:10052E0014508F5E800AE4FDFC7F011214508F5E22
:10053E003001030207897814E6D394B3401408E619
:10054E00944C500EE55E04FFE4FDFC1214508F5ED9
:10055E00D2017814E6C3944C501408E694B3400EBE
:10056E00E55E14FFE4FDFC1214508F5ED201781488
:10057E00E6D394B3500302078908E6D394B350032D
:10058E00020789E4FDFC7F011214508F5ED2010236
:10059E0007897815E6C3944C5002C201301303024A
:1005AE000789E52324F8601624FC602024087026B1
:1005BE00E55E04FFE4FDFC1214508F5E8018E55ECC
:1005CE0014FFE4FDFC1214508F5E800AE4FDFC7FE4
:1005DE00011214508F5E3001030207897815E6D39D
:1005EE0094B3500302078918E6D39406500302070A
:1005FE0089752701E527900E7593FF7814E6D39F32
:10060E00400AE52795505004052780E8E4FDFCAF2D
:10061E00271214508F5ED20102078930130302078E
:10062E0089E52324F8601724FC602224087029E54C
:10063E005E04FF7D017C001214508F5E801AE55E11
:10064E0014FF7D017C001214508F5E800B7D017CA7
:10065E00007F011214508F5EE529452860030207C2
:10066E006FE55824FE602C14604D14607A147003EC
:10067E0002072B24046003020762E55E65507003D7
:10068E00020762E55E04FF7D017C001214508F5E4E
:10069E00020762E5566010E55E04FF7D017C0012E4
:1006AE0014508F5E020762E55E14FF7D017C00121E
:1006BE0014508F5E02076230020FE55E04FF7D016B
:1006CE007C001214508F5E800DE55E14FF7D017C60
:1006DE00001214508F5EE55EB55002C202E55E64F4
:1006EE00017071D202806DE5566010E55E2402FF46
:1006FE007D017C001214508F5E8059E55EB4010DB1
:10070E007D017C00E4FF1214508F5E8047E55E246D
:10071E00FEFF7D017C001214508F5E803730021078
:10072E00E55E2402FF7D017C001214508F5E800E68
:10073E00E55E24FEFF7D017C001214508F5EE550B5
:10074E0024FEFFE55ED39F4002C202E55EC3940223
:10075E005002D202E55175F00AA485F028F52980E1
:10076E001AE5291529700215288010755E01E556C7
:10077E0024FF9204E4FD7FB0122B08E5576403605A
:10078E0004E55770097F0A7E00120003801BE4F512
:10079E0027C3740295272461F8E6FDAF271233C8EC
:1007AE000527E527C3940240E830133B30FF38E5B8
:1007BE005E6401701D300F0B7B05FAFD7FB01225B4
:1007CE00BF8009E4FBFAFD7FB01225BF300E031285
:1007DE001C9FC2133014097D64AF52121E779214FF
:1007EE007D147F031231BEE524600415248005C2FA
:0907FE0003123424C29702018B9E
:0108070022CE
:030000000227686C
:0C276800787FE4F6D8FD7581840227AF6D
:1011E200E709F608DFFA8046E709F208DFFA803EEF
:1011F20088828C83E709F0A3DFFA8032E309F608DC
:10120200DFFA8078E309F208DFFA807088828C8343
:10121200E309F0A3DFFA806489828A83E0A3F608F7
:10122200DFFA805889828A83E0A3F208DFFA804CD1
:1012320080D280FA80C680D4806980F280338010A8
:1012420080A680EA809A80A880DA80E280CA803311
:1012520089828A83ECFAE493A3C8C582C8CCC58389
:10126200CCF0A3C8C582C8CCC583CCDFE9DEE78059
:101272000D89828A83E493A3F608DFF9ECFAA9F0D8
:10128200EDFB2289828A83ECFAE0A3C8C582C8CC2E
:10129200C583CCF0A3C8C582C8CCC583CCDFEADE47
:1012A200E880DB89828A83E493A3F208DFF980CCA9
:1012B20088F0EF60010E4E60C388F0ED2402B404A2
:1012C2000050B9F582EB2402B4040050AF23234549
:0612D2008223901232732A
:1012D800BB010689828A83E0225002E722BBFE0214
:0912E800E32289828A83E4932247
:1012F100BB010689828A83F0225002F722BBFE01DC
:02130100F322D5
:10130300EF8DF0A4A8F0CF8CF0A428CE8DF0A42EFE
:02131300FE22B8
:10131500BC000BBE0029EF8DF084FFADF022E4CCBC
:10132500F875F008EF2FFFEE33FEEC33FCEE9DEC85
:10133500984005FCEE9DFE0FD5F0E9E4CEFD22EDCB
:10134500F8F5F0EE8420D21CFEADF075F008EF2F15
:10135500FFED33FD4007985006D5F0F222C398FD06
:051365000FD5F0EA22A3
:10136A00C2D5EC30E709B2D5E4C39DFDE49CFCEE9E
:10137A0030E715B2D5E4C39FFFE49EFE121315C3EE
:10138A00E49DFDE49CFC800312131530D507C3E4E9
:06139A009FFFE49EFE220D
:1013A000EB9FF5F0EA9E42F0E99D42F0E89C45F0A3
:0113B000221A
:1013B100E493FC740193FD740293FE740393FF2282
:100E8600E547243BF8E60547227838300C02783BE4
:100E9600E475F00112141A0212D82005EB7F2ED247
:100EA600058018EF540F2490D43440D4FF30090B3A
:100EB600EF24BFB41A0050032461FFE54860021511
:100EC60048054BE54B7002054A300C0D7838E47541
:100ED600F00112141AEF0212F10232F87403D20C66
:100EE6008003E4C20CF5478B388A39893AE4F54821
:100EF600F54AF54BE54860077F20120EC180F5756F
:100F060049FFC206C205C207C208C20AC20BC20D09
:100F1600120E8FFF700D300C057F00120ED2AF4BF4
:100F2600AE4A22B4255FC2D5C209120E8FFF24D065
:100F3600B40A00501A75F00A784830D50508B6FF8D
:100F46000106C6A426F620D5047002D20880D9244C
:100F5600CFB41A00EF5004C2E5D2090210D2D2066D
:100F660080C6D20580C0D20780BCD2D580BAD20A4C
:100F760080B47F20120EC12007077401B5480040D7
:100F8600F1120E86FF120EC1020EFAD20DD20B809E
:100F960095120E86FB120E86FA120E86F94A4B70D1
:100FA6000679A37A117BFF20072EE548602A7E008A
:100FB6008E827583001213ED60060EEE654970F0A1
:100FC600C2D5EBC0E0EAC0E0E9C0E0EE121119D0EC
:100FD600E0F9D0E0FAD0E0FB1212D8FF60AAEBC02D
:100FE600E0EAC0E0E9C0E0120EC1D0E02401F9D089
:100FF600E03400FAD0E0FBE5490460DCD549D9804D
:10100600877BFF7A117915D207809C791080027947
:1010160008C20BC20D8008D2D5790A8004790AC2AB
:10102600D5E549047002F549E4FAFDFEFF120E8685
:10103600FC7B08200613120E86FD7B1030050A1273
:101046000E86FE120E86FF7B20EC3382D592D5509B
:1010560013C3E43005069FFFE49EFEE42006039DCD
:10106600FDE49CFCE4CBF8C206EC700CCFCECDCCF4
:10107600E824F8F870F38017C3EF33FFEE33FEED84
:1010860033FDEC33FCEB33FB994002FB0FD8E9EB65
:10109600300605F8D0E0C448B206C0E00AEC4D4E72
:1010A6004F78207B0070C2EAB5490040BCC0E01210
:1010B600111BD0F0D0E0200604C4C0E0C4B206C0C4
:1010C600F0120EAAD0F0D5F0EB020EFA12142A0F87
:1010D60097531011580F684C0F644210154F101D8E
:1010E60044101D490F7D4310235510074610074530
:1010F60010074711C3500F6C2D0F702E0F932B0F37
:1011060074230F912011B12A0F2C4800000F8B3F3A
:101116003F3F00790AA2D5200814300A09B9100207
:101126000404B9080104A2D5200B025001042007CB
:05113600689207B548B6
:10113B00005034C0E07F203008197F30A207720BBB
:10114B00720A500F121172C207C20BC20AC20D7F74
:10115B0030800F300A03E9C0E0120EC1300A03D011
:10116B00E0F9D0E0B548CC300A177F30B9100C123B
:10117B000EC17F583009077F788003B90803120E20
:10118B00C13007057F2D020EC17F20200DF87F2B6C
:10119B00200BF322920780CF286E756C6C29002DE3
:1011AB0050434958D206120E863006F8C2067848CC
:1011BB0030D50108F6020F2C120E862403B405005D
:1011CB004001E49011AA93120EB2743A120EB2D2ED
:0711DB000875480402101121
:10341200C3EE6480948040028007C3E49FFFE49E71
:02342200FE2288
:1013C100EF4E6012EF60010EEDBB010B89828A8343
:1013D100F0A3DFFCDEFA2289F05007F709DFFCA950
:0C13E100F022BBFEFCF309DFFCA9F022A7
:1027740002004EE493A3F8E493A34003F68001F22D
:1027840008DFF48029E493A3F85407240CC8C33366
:10279400C4540F4420C8834004F456800146F6DF35
:1027A400E4800B01020408102040809033E3E47EAF
:1027B400019360BCA3FF543F30E509541FFEE4932A
:1027C400A360010ECF54C025E060A840B8E493A3F1
:1027D400FAE493A3F8E493A3C8C582C8CAC583CA1C
:1027E400F0A3C8C582C8CAC583CADFE9DEE780BED4
:0133FA0000D2
:1013ED00BB010CE58229F582E5833AF583E02250B5
:1013FD0006E92582F8E622BBFE06E92582F8E222FF
:0D140D00E58229F582E5833AF583E4932218
:10141A00FAE6FB0808E6F925F0F618E6CA3AF622D3
:10142A00D083D082F8E4937012740193700DA3A351
:10143A0093F8740193F5828883E473740293686065
:06144A00EFA3A3A380DF65
:1032F800EFB40A07740D123303740A309811A899B1
:10330800B8130CC2983098FDA899C298B811F63035
:0733180099FDC299F599220D
:00000001FF
